:020000040000FA
:10000000012BAD01AC01AE01AD10A90100309E0085
:1000100005309F007C22A92200309E0084309F0082
:100020007C2204309E0080309F007C2220309E0085
:100030009F017C220F309E00F0309F007C220B300D
:100040009E000F309F007C220D309E000F309F00DD
:100050007C2209309E0050309F007C2207309E0099
:10006000D6309F007C224D2227309E0001309F0019
:100070007C2205309E0002309F007C2200309E00D2
:100080008C309F007C2207306B22A70007309E0037
:100090009F017C2227089F007C2A2A306B22A60021
:1000A000261F0800A61E0800E62212308400043035
:1000B0009B0029309E008422672A06306B22A7000D
:1000C000271F68280C306B22A7002718B2280800C9
:1000D000271D72280A306B22A70027182229A7188B
:1000E0004D280800271E7A280E306B22A700271AF9
:1000F000442A0800A71C080008306B22A700271F0D
:100100009A2805309E0000309F007C2204309E001B
:1001100080309F007C2220309E009F017C224D2257
:1001200027309E0001309F007C2205309E00023067
:100130009F007C2A271EA62809309E00C0309F0001
:100140007C2205309E0003309F007C2AA71F0800F8
:1001500009309E0050309F007C2205309E00023006
:100160009F007C2A26306B22A500251F19293030DC
:10017000840008309B0025309E00712254224D22BD
:100180002030A42230086039031D10293108063AB6
:10019000031DCC284D2112293108013A031DD22814
:1001A000342112293108083A031DDC2821309E0031
:1001B00029089F007C2212293108003A031DE228F9
:1001C000C521122931080A3A031DEB2821309E006F
:1001D0009F017C2212293108053A031DFC2820309A
:1001E0009E0040309F007C2204309E003208803800
:1001F000A8009F007C2212293108093A031D022918
:10020000FB2112293108033A031D0829152212295E
:1002100031080B3A031D10293208003A031912293C
:1002200020309F2223309E0005309F007C222E101C
:100230000800AD1C1D29AD104D2227309E00013055
:100240009F007C2A22306B22A600261F3329A61E7F
:1002500033294D22AD1C2E292C22562A27309E00F0
:1002600001309F007C2A080030080339023A031D40
:1002700008003408AF002F080F39AF00003A031D03
:1002800045292030A4222C1008002F08013A031D14
:1002900008002830A422AC100800AD143308A200D6
:1002A0002208013A031D5829A3011230A400B929DC
:1002B0002208023A031D61291230A3006830A4000D
:1002C000B9292208213A031D6A292430A3002D30C0
:1002D000A400B9292208223A031D73293430A3004F
:1002E0006830A400B9292208043A031D7C291B3078
:1002F000A3002430A400B9292208033A031DB7291A
:1003000032088000003A031D8A296830A3006C304F
:10031000A400B9293208013A031D93296C30A300C7
:100320007A30A400B9293208023A031D9C297A3098
:10033000A300A030A400B9293208033A031DA5295F
:10034000A030A300AE30A400B9293208043A031D3E
:10035000AE29AE30A300B430A400B9293208053A62
:10036000031DB729B430A300BA30A400B929A301F2
:10037000A4013708031DC4292308240236020318E8
:10038000C42936082307A4002C2A30080339AF00FB
:10039000003A031DD12921309E0001309F007C22AC
:1003A000E4292F08013A031DDA2921089E009F0144
:1003B0007C22E4292F08023A031DE4293408AF0007
:1003C0002F080F39AF00E82121309E009F017C2AC1
:1003D000AF0A9C0103149C0DAF0BEB292C089C0564
:1003E0000319F72921309E0001309F007C2A21301B
:1003F0009E009F017C2A3208A900003A0319112AA5
:10040000AE01AC01522228309E0011309F007C22A8
:10041000E6221230840004309B0029309E008422A2
:10042000672A28309E009F017C2A30080339023A4F
:10043000031D080034080F39B400003A031D242AB4
:1004400020309F222C1408003408013A031D0800B4
:1004500028309F22AC14080008309B002308240297
:10046000083C031C382A23082402031908009B00B7
:100470002130C03885118F22230815238F22A30A2B
:100480009B0B3C2A85150800AD1C0800AD104D22C1
:1004900027309E0001309F007C2A23309E000830C8
:1004A0009F007C2A2B304E2A27304E2A23309E0074
:1004B00001302E1804389F007C220130AE0608005F
:1004C0002B309E000330AE1804389F007C2A602237
:1004D0000230AE06080085118F2203018F22851598
:1004E000080085111E088F221E088F228000840AB2
:1004F0009B0B742A8515080085111E0880388F22F1
:100500001F088F228515080085111E08C0388F220C
:1005100000088F22840A9B0B882A85150800A000FA
:100520000830A100A00D85100318851405142010B3
:10053000051920140510A10B922A200808009E001E
:100540006B2280179F007C2A9E006B2280139F00E5
:100550007C2AFA309D00AF229D0BAB2A08009C013B
:100560009C0BB02A080006083F3991000800920150
:1005700093019401950103301105031DC12A121541
:10058000C52A911C9214111C12140C301105031968
:10059000D82A0F08911D9307111D930230301105C1
:1005A000031908000F08111E9402911E94070800F9
:1005B00002308D068D1C080030301105031908002B
:1005C0000130111E9507911E95020800B3221109F2
:1005D0003C3903198E01100811043C3A3C39031DC3
:1005E000F32A8E01F72A0C300E02031C8E0A033008
:1005F0000E02031C00308F0002308F07110890009C
:10060000B72A8316873081008B01143085003F3074
:10061000860083120830850001308F003F30900043
:100620008E010120051A5D20122B9A0003308A00EA
:100630001A088207123401341034013400340034B3
:1006400000340834DA34083481340334013400349B
:1006500001340234033401340934023422340034C6
:100660000134013404348034323409340434013424
:1006700000340134033401340234053409342134A4
:10068000003401340034013422343434003407346B
:1006900005348134033404340034323405340134F5
:1006A00009340234A134013409340134A134003452
:1006B0000534093419340134293403341534003431
:1006C00025340134953403347534013481340234D3
:1006D00095340134753405348134013405340134E2
:1006E0000934303409343134093438341534813420
:1006F00025347F347534083495340334813406341A
:10070000C034C03404340334093404340E340334A4
:100710004A3400344A340034313400344F34003425
:10072000443400344D340034263403344A34003425
:100730004F340034593400345034003441340034E0
:100740004434003420340034573400344834003406
:1007500045340034453400344C3400342034003403
:100760004D3400344F3400345534003453340034A5
:10077000453400340E3403344A34003457340034E2
:100780004D340034303400343034003431340034EB
:100790000634033442340034613400340634033404
:0807A0003134003470340034E0
:02400E00F33F7E
:00000001FF
